:1000000010C01FC01EC01DC01CC01BC01AC019C01C
:1000100018C017C016C015C014C013C012C011C03C
:1000200010C011241FBECFE5D1E0DEBFCDBF10E070
:10003000A0E6B0E001C01D92A836B107E1F7B6D046
:10004000A5C1DECFFC011082CF9BFECF8CE18A954B
:10005000F1F7000088E38A95F1F700C0CF9903C05B
:1000600080818160808388E38A95F1F700C0CF9911
:1000700003C080818260808388E38A95F1F700C0A5
:10008000CF9903C080818460808388E38A95F1F7EB
:1000900000C0CF9903C080818860808388E38A95FF
:1000A000F1F700C0CF9903C080818061808388E32D
:1000B0008A95F1F700C0CF9903C080818062808368
:1000C00088E38A95F1F700C0CF9903C080818064EE
:1000D000808388E38A95F1F700C0CF9903C08081BF
:1000E0008068808388E38A95F1F700C08CE18A9567
:1000F000F1F700000895DE9A98E39A95F1F700C0B1
:10010000282F332727FD309520FF02C0DE9801C03D
:10011000DE9A98E39A95F1F700C021FF02C0DE98BD
:1001200001C0DE9A98E39A95F1F700C022FF02C061
:10013000DE9801C0DE9A98E39A95F1F700C023FF9C
:1001400002C0DE9801C0DE9A98E39A95F1F700C0EC
:1001500024FF02C0DE9801C0DE9A98E39A95F1F779
:1001600000C025FF02C0DE9801C0DE9A98E39A9590
:10017000F1F700C026FF02C0DE9801C0DE9A98E3C6
:100180009A95F1F700C087FF02C0DE9801C0DE9AA1
:1001900088E38A95F1F700C0DE9898E39A95F1F725
:1001A00000C088E38A95F1F700C008958F929F926E
:1001B000AF92BF92CF92DF92EF92FF920F931F9375
:1001C000CF93DF9380E886BD16BCDE98D698D8988A
:1001D000D09ADB98D39ADD98D59A1092650000E00A
:1001E00010E0C1E0D0E099249A948824839487E6B3
:1001F00090E028DF80916700873409F060C080912B
:100200006500813059F5D89ADE9AD69ADB9AC017E4
:10021000D10708F04EC0C8018C1B9D0BBE01A2D0B7
:1002200080E090E017C0DD9AE7E8F3E13197F1F75D
:1002300000C00000DD9820E030E008C0E7E8F3E10E
:100240003197F1F700C000002F5F3F4F26173707A7
:10025000A8F301968C179D0730F32BC08F3F49F50B
:10026000D89ADE9AD69ADB98C017D10710F5C80144
:100270008C1B9D0BBE0176D080E090E017C0DD9A0C
:10028000E7E8F3E13197F1F700C00000DD9820E0E6
:1002900030E008C0E7E8F3E13197F1F700C0000073
:1002A0002F5F3F4F26173707A8F301968C179D073E
:1002B00030F3D698DE98D8981092650098CF89359B
:1002C00091F48092650086E690E0BCDE82E690E0E4
:1002D000B9DE83E690E0B6DEB0906200AA24809199
:1002E0006300E50113C08937A1F49092650086E6AA
:1002F00090E0A8DE82E690E0A5DE83E690E0A2DE54
:10030000D0906200CC2480916300E601C80FD11D1B
:100310006ECF843591F486E690E094DE80E690E03E
:1003200091DE81E690E08EDEF0906000EE24809118
:1003300061008701080F111D5ACF86E690E082DE2A
:100340001092640008C087E690E07CDE8091640033
:100350008F5F80936400909164008091660098178D
:1003600094F345CFAA1BBB1B51E107C0AA1FBB1FBB
:10037000A617B70710F0A61BB70B881F991F5A9531
:10038000A9F780959095BC01CD010895F894FFCF11
:00000001FF
